:1000000010C01FC01EC01DC01CC01BC01AC019C01C
:1000100018C017C016C015C014C013C012C011C03C
:1000200010C011241FBECFE5D1E0DEBFCDBF20E060
:10003000A0E6B0E001C01D92AF37B207E1F701D1F1
:100040008EC1DECFDC01FA0110828C918623E9F7A4
:100050008CE18A95F1F7000088E38A95F1F700C0FA
:100060008C91862319F080818160808388E38A9552
:10007000F1F700C08C91862319F080818260808323
:1000800088E38A95F1F700C08C91862319F080816E
:100090008460808388E38A95F1F700C08C91862381
:1000A00019F080818860808388E38A95F1F700C029
:1000B0008C91862319F080818061808388E38A9502
:1000C000F1F700C08C91862319F0808180628083D3
:1000D00088E38A95F1F700C08C91862319F080811E
:1000E0008064808388E38A95F1F700C08C91862331
:1000F00019F080818068808388E38A95F1F700C0D9
:100100008CE18A95F1F700000895FC019081862F1B
:1001100080959823908398E39A95F1F700C0908199
:1001200040FF02C0962B01C09823908398E39A95D4
:10013000F1F700C0908141FF02C0962B01C09823C7
:10014000908398E39A95F1F700C0908142FF02C036
:10015000962B01C09823908398E39A95F1F700C0FD
:10016000908143FF02C0962B01C09823908398E3AF
:100170009A95F1F700C0908144FF02C0962B01C010
:100180009823908398E39A95F1F700C0908145FFFA
:1001900002C0962B01C09823908398E39A95F1F7BB
:1001A00000C0908146FF02C0962B01C09823908327
:1001B00098E39A95F1F700C047FF04C08081862B31
:1001C000808303C090819823908388E38A95F1F718
:1001D00000C08081862B808398E39A95F1F700C058
:1001E00088E38A95F1F700C00895FF920F931F935B
:1001F000CF93DF938C01F62EEA0110927E001092CD
:100200007D00E0917D00F0917E00EC0FFD1F4081AC
:100210006F2DC8017ADF20917D0030917E002F5F25
:100220003F4F30937E0020937D00FE01E20FF31FCD
:1002300080818111E6CFDF91CF911F910F91FF90C7
:10024000089580E886BD16BCD99AD19A82E087B914
:1002500084E886B982E0E82E93E0D92E04E610E027
:10026000CAE0D0E020E2F22EE7B8369A3699FECF07
:1002700084B195B190937C0080937B00D7B8369A77
:100280003699FECF24B135B130937A0020937900AE
:10029000E0917B00F0917C00CF01B80139D0CB0117
:1002A000BE0136D0805D80936000CF01BE0130D0AA
:1002B000482FCB01BE012CD0805D80936100405D52
:1002C00040936200F0926300C901B80121D0CB01D4
:1002D000BE011ED0805D80936400C901BE0118D0AC
:1002E000282FCB01BE0114D0805D80936500205D76
:1002F000209366001092670040E650E062E08BE3D6
:1003000090E073DF4AE062E08BE390E0FEDEACCF8A
:1003100097FB072E16F4009406D077FD08D00BD07B
:1003200007FC05D03EF4909581959F4F08957095F8
:1003300061957F4F0895AA1BBB1B51E107C0AA1FFF
:10034000BB1FA617B70710F0A61BB70B881F991F76
:100350005A95A9F780959095BC01CD010895F89420
:02036000FFCFCD
:00000001FF
